:10094A0000C000F900A400B000990092008200F8EB
:10095A00008000900088008300C600A10086008EF7
:0A0BCA00E51125E0F511EF421122BC
:0D0B4D00E51125E0F511EFF45401421122ED
:040C4200EF5211223A
:070BFF00EFF4540152112232
:040C4600EF42112246
:070C0600EFF454014211223A
:0E0B2300E511F45401FFE51154FE4FF51122C7
:060C3000E5115401FF2252
:0D0B5A00E511C313FFE51154015FF51122F1
:0D0B6700E511C313FFE51154014FF51122F4
:040A1500135401FD78
:0E0A1900E51125E0F511EDF45F5401421122C4
:0E0B3100E51125E0F511EFF45D5401421122AB
:08000300EDF45F5401521122DB
:080BE700EFF45D5401521122EC
:080BEF00EDF45F5401421122F4
:080BF700EFF45D5401421122EC
:070C0D00EDF45F5401FF222A
:070C1400EFF45D5401FF2223
:0D0B7400E51825E0FFE51154014FF51822AA
:0D0B8100E5185401FFE51154FE4FF5112257
:100A0200E5185401FFE51154FE4FF511E518C31323
:030A1200F51822B2
:100B04008E5E8F5FE55F2DFFE55E3C8FF0020496FD
:100A27008E608F61C3E5619DFFE5609C8FF00204D6
:010A37009628
:090BDE001203D5EE8FF00204961B
:0F0B14008B5B8A5C895D1203E7EE8FF00204961B
:070C1B00E475F00102045E24
:070C220074FFF5F002045E0F
:100A38008E628F63E5625CFFE5635DCF8FF0020431
:010A48009617
:100A49008E648F65E5644CFFE5654DCF8FF0020438
:010A59009606
:100A5A008E668F67E5666CFFE5676DCF8FF00204DF
:010A6A0096F5
:100A6B00EFF4FFEEF4FEEF2401FFE43E8FF00204FF
:010A7B0096E4
:060C3600EFF45401FF225F
:060C3C00EE8FF0020496A9
:0A0BD400EFF4FFEEF48FF002049638
:1008F4008B4B8A4C894D120433FFAEF0AB4EAA4F9A
:10090400A950120433FDAB4BAA4CA94DE5F08DF070
:0F091400120496AB4EAA4FA950EE8FF002049634
:1005E3008E528F538B548A5589567C037DE81203B0
:1005F300E7EFC454F07B00FAAE52AF537C037DE8BF
:100603001203E78C528D53AE52AF537C007D6412BC
:1006130003E7EFFEE4EE4202AE52AF537C007D648B
:100623001203E78C528D53AE52AF537C007D0A12F6
:1006330003E7EFC4F8540FC868FFEEC454F048FE54
:10064300EFFBEE4202AE52AF537C007D0A1203E78A
:100653008C528D53E5524AFFE5534BAB54AA55A92F
:0706630056CF8FF002049650
:1006E9008E578F58E558780CCEA2E713CE13D8F859
:1006F9007E00540FFF7C037DE81203D58E598F5A73
:10070900E557FF3395E07E00EF540FFF7C007D64D1
:100719001203D5EF255AF55AEE3559F559E558AE74
:10072900577804CEA2E713CE13D8F87E00540FFFF2
:100739007C007D0A1203D5EF255AF55AEE3559F595
:1007490059E558540F255AF55AE43559F559855A3A
:04075900F002049610
:10096A00E51125E0F511C3EF9DEC6480F8EE648093
:0B097A00984004431101225311FE229B
:10098500E51125E0F511D3EF9DEC6480F8EE648068
:0B099500985004431101225311FE2270
:1009A000E51125E0F511D3EF9DEC6480F8EE64804D
:0B09B000984004431101225311FE2265
:1009BB00E51125E0F511C3EF9DEC6480F8EE648042
:0B09CB00985004431101225311FE223A
:1009D600E51125E0F511EF6D7002EE6C6004431130
:0609E60001225311FE2264
:1009EC00E51125E0F511EFB50508EEB5040443114A
:0609FC0001225311FE224E
:100A7C00C3EF9DEC6480F8EE64809850035311FE34
:010A8C002247
:100A8D00D3EF9DEC6480F8EE64809840035311FE23
:010A9D002236
:100A9E00D3EF9DEC6480F8EE64809850035311FE02
:010AAE002225
:100AAF00C3EF9DEC6480F8EE64809840035311FE11
:010ABF002214
:0C0B8E00EFB50507EEB504035311FE227D
:0C0B9A00EF6D7002EE6C60035311FE2240
:100AC000C3EF9DEC6480F8EE64809840034311010D
:010AD0002203
:100AD100D3EF9DEC6480F8EE6480985003431101DC
:010AE10022F2
:100AE200D3EF9DEC6480F8EE6480984003431101DB
:010AF20022E1
:100AF300C3EF9DEC6480F8EE6480985003431101CA
:010B030022CF
:0C0BA600EF6D7002EE6C60034311012241
:0C0BB200EFB50507EEB504034311012266
:070C2900E4FF0FBF0AFC22EB
:1008C400E4FEC2B4120C29C2B3120C29D2B3120C26
:1008D40029D2B4120C29E4FDEE25E0FE3094034342
:1008E4000601C2B3120C29D2B30DBD08EBAF062228
:1001F4000510E510C394054003E4F510E510146000
:100204005B1470030202B01470030202FC24036046
:100214000302034E7C0090000DE0540FFD25E0FF27
:10022400EC33FE744A2FF58274093EF583E493FCA3
:10023400740193FD43040890010AE0FFC4131313EF
:10024400540130E0057DFF0203A4EF131313541F80
:1002540020E0030203A453057F0203A490000CE0F2
:10026400FEA3E07804CEA2E713CE13D8F87C0054A2
:100274000FFD25E0FFEC33FE744A2FF58274093E2E
:10028400F583E493FC740193FD43040490010BE0B3
:1002940030E0057DFF0203A490010AE0FFC4540F7F
:1002A40020E0030203A453057F0203A490000CE0A2
:1002B400FF3395E07C00EF540FFD25E0FFEC33FEA7
:1002C400744A2FF58274093EF583E493FC74019318
:1002D400FD43040290010BE0FFC31330E0057DFFF2
:1002E4000203A490010AE0FFC413540720E00302B0
:1002F40003A453057F0203A490000CE0FEA3E0785E
:100304000CCEA2E713CE13D8F87C00540FFD25E0E1
:10031400FFEC33FE744A2FF58274093EF583E493AF
:10032400FC740193FD43040190010BE0FF1313548B
:100334003F30E0047DFF806890010AE0FFC413139E
:10034400540330E05B53057F805690010BE0F9C401
:100354001313540175F008A4FBAAF0E9C413131392
:10036400540175F010A4FFE5F04AFAEF4BFBE9C421
:1003740013540175F004A4FFEA45F0FAEB4FFBE9CE
:10038400C4540125E0FFE4334AFEEB4FFFE91313A5
:10039400135401FBEEEF4BF4FFEEF47410FCAD07C5
:1003A4007B10C2B3120C29EC20E704C2B78002D23E
:1003B400B7120C29ED25E0FDEC33FCD2B3120C2965
:1003C400DBE0D2B7120C29C2B5120C29D2B5020C4B
:0103D40029FF
:10000E00E52E70030201F3152E0517E517B405173B
:10001E00AF30EFC4135401F45401FFC43354E0FF66
:10002E00E53054DF4FF530E517B40A1CAF30EFC49E
:10003E00135401F45401FFC43354E0FFE53054DF90
:10004E004FF530051DE4F517E4F552E55213131381
:10005E00541F2412F8E6FD7C00E5525407FF74018C
:10006E007E00A807088005C333CE33CED8F9FFEE45
:10007E005CFEEF5D4E6043E55225E025E0246EF513
:10008E0082E43400F583E0FEA3E0FFE55225E0258F
:10009E00E0246CF582E43400F583E0FCA3E0C39F1A
:1000AE00EC9E5016E55225E025E0246CF582E434F2
:1000BE0000F583E475F00112041DE55225E025E0FC
:1000CE00246EF582E43400F583E0FEA3E0FFE552F2
:1000DE0025E025E0246CF582E43400F583E0FCA3F2
:1000EE00E0C39FEC9E407AE55225E025E0246CF5B6
:1000FE0082E43400FEC3E582946CFFEE9400FE7C35
:10010E00007D021203E77C007D021203E77C007D76
:10011E00081203E7741E2FF8C000E6FFC007E55271
:10012E0025E025E0246CF582E43400FEC3E58294DC
:10013E006CFFEE9400FE7C007D021203E77C007DD6
:10014E00021203E77C007D081203E7AF057401A8D5
:10015E0007088002C333D8FCFED0E04ED000F680F4
:10016E0079E55225E025E0246CF582E43400FEC3E7
:10017E00E582946CFFEE9400FE7C007D021203E794
:10018E007C007D021203E77C007D081203E7741EDB
:10019E002FF8C000E6FFC007E55225E025E0246CED
:1001AE00F582E43400FEC3E582946CFFEE9400FE0B
:1001BE007C007D021203E77C007D021203E77C00C7
:1001CE007D081203E7AF057401A807088002C33348
:1001DE00D8FCF4FED0E05ED000F60552E552642065
:0601EE006003020059222B
:10080A00E51DB41E19AF30EFC413135401F454019B
:10081A00FFC4333354C0FFE53054BF4FF530E51DF4
:10082A00B43C1CAF30EFC413135401F45401FFC499
:10083A00333354C0FFE53054BF4FF530E4F51D2281
:03000B0002075D8C
:10075D00C0E0C0D075D008758CEEAF30EF13131319
:10076D005401F45401FF33333354F8FFE53054F79B
:10077D004FF530053AE53A30E0020516E53AB40A90
:10078D0015AF30EFC45401F45401FFC454F0FFE52C
:10079D003054EF4FF530E53AB4141AAF30EFC4547E
:1007AD0001F45401FFC454F0FFE53054EF4FF53020
:0A07BD00052E753A00D0D0D0E032CE
:1007C7007594FF752F05E4F530F53190000CF0A313
:1007D700F090010BE054F7F054EFF054DFF054BF02
:1007E700F0547FF090010AE054F7F054EFF054DF33
:1007F700F054BFF0547FF0A3E054FEF054FDF054E2
:03080700FBF022E1
:040C4A00752F0922D7
:10084A00E4FFEF25E025E0246CF582E43400F5832B
:10085A00E4F0A3F00FBF20EAE4FF7F4090002CE40D
:10086A00F0A3DFFCE4FF741E2FF8E4F60FBF04F6D2
:0D087A00E4FF74192FF8E4F60FBF04F62216
:0E0B3F00758911D2B4D2B9D2A9D28CD2AF220C
:10088700AFA0EFC3135455FEEF25E054AA4EFF1354
:10089700135433FEEF25E025E054CC4EFF54F0FE11
:1008A700E590540F4EF4F522EF540FF4540FF5234F
:0D08B7001208C4EFF4F5248528800201F436
:10066A00E4FF74222FF8E6FE743F2FF8A6060FBFA8
:10067A0006F0E4FF74282FF8E6FE74452FF8A60664
:10068A000FBF06F0E4FF74682FF8E6FE74202FF51A
:10069A0082E43401F583EEF00FBF20EAE4FF74EC44
:1006AA002FF582E43400F583E0FE74402FF582E4EE
:1006BA003401F583EEF00FBF20E4E4FF741E2FF837
:1006CA00E6FE74362FF8A6060FBF04F0E4FF74198D
:0F06DA002FF8E6FE74322FF8A6060FBF04F022A9
:100923007551011207C712084A120B3F12088712AA
:10093300050A12000E12080A12066AE55160EDE478
:07094300F551120C4A80E59A
:10050A00AF2FEF13135401FF120BCAE51130E007A6
:10051A00E490010CF0A3F0E5225401FFE53F5401F9
:10052A00FD120A19E51130E0097B017A01790C12F2
:10053A000C1BAF22EFC3135401FFAE3FEEC3120AE6
:10054A0015E51130E0097B017A01790C120C22AF12
:10055A0022EF13135401FFAE3FEE13120A15E511F1
:10056A0030E007E490010CF0A3F0E52F5401FF12EC
:10057A000BCA120B74E51130E00F90010CE0FEA3D8
:10058A00E0FF7D107C27120B9AE51130E007E4901A
:10059A00010CF0A3F0120B81E51130E00F90010C71
:1005AA00E0FEA3E0FF7D107C27120A9EE51130E0F1
:1005BA000D7B017A01790C7F0F7E27120C3C120AFF
:1005CA0002E51130E01190010CE0FEA3E0FF7B018F
:0905DA007A00790C1205E30022FD
:03000000020BBE32
:0C0BBE00787FE4F6D8FD758187020923DA
:1003D500EF8DF0A4A8F0CF8CF0A428CE8DF0A42E3C
:0203E500FE22F6
:1003E700C2D5EC30E709B2D5E4C39DFDE49CFCEE31
:1003F70030E715B2D5E4C39FFFE49EFE1204B5C3F0
:10040700E49DFDE49CFC80031204B530D507C3E4EA
:060417009FFFE49EFE229F
:10041D00C5F0F8A3E028F0C5F0F8E582158270026A
:06042D001583E038F02207
:10043300BB010A89828A83E0F5F0A3E02250068794
:10044300F009E71922BBFE07E3F5F009E319228956
:0B045300828A83E493F5F07401932289
:10045E00BB010789828A8302041D500B09C5F02750
:10046E00F7C5F01937F722BBFE0D09F8E325F0F3B7
:10047E00C5F019E338F322F889828A837401932533
:08048E00F0C5F0F8E4933822F8
:10049600BB010A89828A83F0E5F0A3F0225006F7B1
:0F04A60009A7F01922BBFE06F3E5F009F31922AE
:1004B500BC000BBE0029EF8DF084FFADF022E4CC2B
:1004C500F875F008EF2FFFEE33FEEC33FCEE9DECF4
:1004D500984005FCEE9DFE0FD5F0E9E4CEFD22ED3A
:1004E500F8F5F0EE8420D21CFEADF075F008EF2F84
:1004F500FFED33FD4007985006D5F0F222C398FD75
:050505000FD5F0EA2211
:00000001FF
